:0200000480007A
:100000006F004005732F2034930F8000630AFF03B5
:10001000930F90006306FF03930FB0006302FF038A
:10002000170F0000130F4F2963040F0067000F0024
:10003000732F203463540F006F00400093E19153FD
:10004000171F000023203FFC171F0000232E0FFA6C
:100050006FF01FFF930000001301000093010000E8
:10006000130200009302000013030000930300003A
:100070001304000093040000130500009305000022
:10008000130600009306000013070000930700000A
:1000900013080000930800001309000093090000F2
:1000A000130A0000930A0000130B0000930B0000DA
:1000B000130C0000930C0000130D0000930D0000C2
:1000C000130E0000930E0000130F0000930F0000AA
:1000D000732540F16310050097020000938202012E
:1000E000739052307350447497020000938202015F
:1000F00073905230735000189702000093824202AE
:10010000739052309B021000939252039382F2FF3D
:100110007390023B9302F0017390023A73504030A7
:100120009702000093824201739052307350203046
:100130007350303093010000970200009382C2ECAC
:1001400073905230130510001315F501635C050020
:100150000F00F00F930110009308D0051305000065
:100160007300000093020000638A02007390521033
:10017000B7B200009B82921073902230735000300F
:10018000372500001B05058073200530970200000D
:100190009382420173901234732540F17300203032
:1001A00093012000972000009380C0E5375134125E
:1001B0001B018167970700009387470123A0200058
:1001C00003A700006F00800013070100B75334122B
:1001D0009B8383676318770A9301300097200000A0
:1001E000938040E237E1BC9A1B0101EF97070000C2
:1001F00093874701A3A0200003A710006F00800091
:1002000013070100B7E3BC9A9B8303EF631C7706D7
:1002100093014000972000009380C0DE37C1ADDE1F
:100220001B01F1EE970700009387470123A12000EF
:1002300003A720006F00800013070100B7C3ADDEE5
:100240009B83F3EE63107704930150009720000026
:10025000938040DB3701EDFE1B0111019707000081
:1002600093874701A3A1200003A730006F008000FF
:1002700013070100B703EDFE9B831301631477009E
:10028000631030020F00F00F6380010093911100A2
:1002900093E111009308D00513850100730000005D
:1002A0000F00F00F930110009308D0051305000014
:1002B000730000009302600073232034E39462FC17
:1002C0007390173473002030731000C000000000DA
:1002D000000000000000000000000000000000001E
:1002E000000000000000000000000000000000000E
:1002F00000000000000000000000000000000000FE
:1010000000000000000000000000000000000000E0
:1010100000000000000000000000000000000000D0
:1010200000000000000000000000000000000000C0
:1010300000000000000000000000000000000000B0
:081040000000000000000000A8
:1020000000000000000000000000000000000000D0
:040000058000000077
:00000001FF
